:020000040000FA
:0600000060283F300130D2
:08000800A000030EA100831209
:1000100005191028831601178312B2308100422877
:100020008316011383120B191C28AE17280A031913
:100030002E17AE192D283B28AE13AE192A282E1FD5
:100040003B28AE1A3B28A701A601A501A801AE01D5
:10005000AE164228F030AE0542282D152E13AE12F2
:100060002708AB002608AA002508A9002808AC002C
:10007000F030AE0542282E0DA80DA50DA60DA70D3A
:10008000AE1AAE0A8B100B11210E8300A00E200EAB
:02009000090065
:1000C000203084008001840A80300402031C6228EE
:1000D000F82183160C30850587018312850187017D
:1000E0000730990000309A00103083168E0083127A
:1000F000603083168F0083120030831691009F00BA
:100100008312C83083168100831231309000003092
:1001100083168C00831210308B003D1BBE013D1BEB
:10012000BF013D1F232281018E018F010B118B1016
:100130000B108C018B17AB202D19AD20CA21B30BEE
:10014000A928031085190314BA0DF0303A020319D7
:10015000422124229B2864000800A91F2D11A91FF9
:100160000800291B2D11291B08002B082A06290627
:100170002C02031D2D11031D08002D110130B700A5
:100180008B132030370783169B001C141A08831228
:10019000A4001030370783169B001C141A08831222
:1001A000A3000030370783169B001C141A08831223
:1001B000A2008B1724082B02031D3C2923082A02C6
:1001C000031D3C2922082906F039A91EE039031D28
:1001D0003C29220829050F39031912290130370259
:1001E000031DF7283E18F7283E14AD1707220230EA
:1001F0003702031D0029BE180029BE14AD170A22BC
:1002000003303702031D09293E1909293E15AD1790
:100210000D2204303702031D1229BE191229BE1502
:10022000AD171022290922050F3903193C29013085
:100230003702031D20293E1C20293E10AD17132232
:1002400002303702031D2929BE1C2929BE10AD1713
:10025000172203303702031D32293E1D32293E1179
:10026000AD171B2204303702031D3B29BE1D3B295D
:10027000BE11AD171F223C29B70A053037020318FB
:100280000800C028B601B3019630B4000130B500B3
:100290000130B70085018701AD13AA21AB20B30B54
:1002A0006B29031085190314BA0DF0303A020319B3
:1002B0009A29B41F8501B41F8701B40B6B29370835
:1002C000B6080319B60003196929FF3085008700B5
:1002D000B6039630B4002D1D4E292D11A91F4E29AD
:1002E000291B4E29A91E29120F30290503194E2951
:1002F000B9012918B90AA918B90A2919B90AA919F5
:10030000B90AB9184E2939194E298B1320303707ED
:10031000BC002B08BB00D82110303707BC002A08CE
:10032000BB00D82100303707BC002908BB00D8210A
:100330008B17A42185018701B70AB6010530370262
:10034000031C4E2923220800043037020319080039
:10035000850187011430B90033300F1E85000F1A54
:100360008501FF300F1A87000F1E8701AB202D1D5E
:10037000AC292D11290A0319C129A91FAC29291B50
:10038000AC290F302905031DAA29B90BAC29850119
:1003900087010800AD1F0800AD131030BC003E08F7
:1003A000BB00D8213030BC003F08BB00D82108007A
:1003B0003C088B1383169B001C141A0883128B179E
:1003C0003B02031908008B133B0883161C159A0087
:1003D00083123C0883169B0055309D00AA309D0077
:1003E0009C1464009C18F1291C1183128B170800BF
:1003F000831600309B001C141A088312BD0083165C
:1004000010309B001C141A088312BE000800013033
:10041000BE0008000230BE0008000430BE00080024
:100420000830BE000800850187013E1008008501E4
:100430008701BE100800850187013E110800850173
:100440008701BE11080008008F08031908008F01FA
:1004500003303E0503191C2B02303E05031D5110CD
:100460005408EB3C031805125118392AD40B442ABE
:100470003E2AD4035408C83C031C442A0516F53010
:10048000D4005108013AD10002303E05031DD110BD
:100490005508E63C03188512D118512AD50B5C2A61
:1004A000562AD5035508B93C031C5C2A8516F03042
:1004B000D5005108023AD10002303E05031D51110A
:1004C0005608DC3C031805105119692AD60B742A0A
:1004D0006E2AD6035608B63C031C742A0514E6306F
:1004E000D6005108043AD10002303E05031DD11157
:1004F0005708F03C03188510D119812AD70B8C2A94
:10050000862AD7035708D73C031C8C2A8514FA3057
:10051000D7005108083AD10002303E05031D5112A0
:100520005808E03C03188710511A992AD80BA42ABE
:100530009E2AD8035808C13C031CA42A8714EA3019
:10054000D8005108103AD10006303E05031DD112E3
:100550005908D43C03180711D11AB12AD90BBC2A67
:10056000B62AD9035908A73C031CBC2A0715DE305C
:10057000D9005108203AD10006303E05031D511321
:100580005A08BF3C03180710511BC92ADA0BD42A9A
:10059000CE2ADA035A089C3C031CD42A0714C9301B
:1005A000DA005108403AD10006303E05031DD11350
:1005B0005B08D73C03188712D11BE12ADB0BEC2A1E
:1005C000E62ADB035B08BE3C031CEC2A8716E130FD
:1005D000DB005108803AD10006303E05031D521061
:1005E0005C08F13C031807125218F92ADC0B042BA3
:1005F000FE2ADC035C08CF3C031C042B0716FB30EF
:10060000DC005208013AD20006303E05031DD2102C
:100610005D08E93C03188711D218112BDD0B1C2B48
:10062000162BDD035D08B23C031C1C2B8715F33031
:10063000DD005208023AD2000C303E0503196C2B43
:100640003E1D282B54083C3C031C282B85018701A8
:10065000D40B0800D0034630D4000B305002031DE9
:10066000322B05160A305002031D372B8516093030
:100670005002031D3C2B051408305002031D412B72
:10068000851407305002031D462B87140630500294
:10069000031D4B2B071505305002031D502B07146B
:1006A00004305002031D552B871603305002031DE2
:1006B0005A2B071602305002031D5F2B871501309D
:1006C0005002031D632B12305002031C08008501E9
:1006D00087010C30D000080020303E050319B62BEE
:1006E000D40B772B0508103A85008230D400D50B47
:1006F0007E2B0508203A85007D30D500D60B852B52
:100700000508013A85007330D600D70B8C2B0508FD
:10071000023A85008730D700D80B932B0708023A9E
:1007200087007730D800D90B9A2B0708043A870046
:100730006B30D900DA0BA12B0708013A870056303D
:10074000DA00DB0BA82B0708203A87006E30DB00AD
:10075000DC0BAF2B0708103A87008830DC00DD0B7C
:10076000B62B0708083A87008030DD0040303E0590
:0A0770000319BC2B85018701080066
:084000000600000006000200AA
:02400E00CC33B1
:1042000001008100820084008800B100B200B40087
:10421000B800A100A200FF00FF00FF00FF00FF00A8
:104220000000010001000100010001000100010087
:10423000010001000100FF00FF00FF00FF00FF0080
:10424000010000000000000000000000000000006D
:10425000000000000000FF00FF00FF00FF00FF0063
:104260000000FF00FF00FF00FF00FF00FF00FF0055
:10427000FF00FF00FF00FF00FF00FF00FF00FF0046
:10428000FF00FF00FF00FF00FF00FF00FF00FF0036
:10429000FF00FF00FF00FF00FF00FF00FF00FF0026
:1042A000FF00FF00FF00FF00FF00FF00FF00FF0016
:1042B000FF00FF00FF00FF00FF00FF00FF00FF0006
:1042C000FF00FF00FF00FF00FF00FF00FF00FF00F6
:1042D000FF00FF00FF00FF00FF00FF00FF00FF00E6
:1042E000FF00FF00FF00FF00FF00FF00FF00FF00D6
:1042F000FF00FF00FF00FF00FF00FF00FF00DD00E8
:00000001FF
